:020000040000FA
:04000000DFEF0CF032
:08000800056ED8CF06F0E0CF31
:1000100007F00001E9CF0DF0EACF08F0E1CF09F0D9
:10002000E2CF0AF0D9CF0BF0DACF0CF0F3CF14F017
:10003000F4CF15F0FACF16F000C00FF001C010F0A9
:1000400002C011F003C012F004C013F09DAA2CEFFF
:1000500000F09EBA54EF01F00FC000F010C001F0A4
:1000600011C002F012C003F013C004F00DC0E9FF8C
:1000700008C0EAFF09C0E1FF0AC0E2FF0BC0D9FFD8
:100080000CC0DAFF14C0F3FF15C0F4FF16C0FAFF6E
:10009000055007C0E0FF06C0D8FF1000F2CF0EF0F9
:1000A000F29EB40FF66E000EF7220900F5500EBE58
:1000B000F28E120000000000004444440044AAAA4A
:1000C000000000AAEEAAEEAA66CCCC66EEAA2244F4
:1000D00088AA44AA44AA6644440000004488888848
:1000E00044442222224400AA44AA000044EE4400D0
:1000F00000000044880000EE0000000000004422E0
:1001000022448888EEAAAAAAEE44CC4444EEEE2209
:10011000EE88EEEE22EE22EEAAAAEE2222EE88EE83
:1001200022EECC88EEAAEEEE22448888EEAAEEAA51
:10013000EEEEAAEE2266004400440000440044882B
:10014000224488442200EE00EE008844224488CCF9
:100150002266004444AAEE8866EEAAEEAAAACCAAB9
:10016000EEAACCEE888888EECCAAAAAACCEE88EEBD
:1001700088EEEE88EE8888EE8888AAEEAAAAEEAA13
:10018000AAEE444444EE222222AAEE88AACCCCAAAB
:1001900088888888EEAAEEEEAAAA00CCAAAAAA4469
:1001A000AAAAAA44EEAAEE888844AAAAEE66EEAAF3
:1001B000CCEEAAEE88EE22EEEE44444444AAAAAA6B
:1001C000AAEEAAAAAAAA44AAAAEEEEAA00AA44449F
:1001D000AAAAAA444444EE224488EEEE888888EE17
:1001E0008888442222EE222222EE44AA0000000047
:1001F000000000EE88440000000044AAAA6688CCF3
:10020000AAAACC00668888662266AAAA660044AAC2
:10021000CC666644EE44440044AA66CC88CCAAAAC4
:10022000AA440044444444004444888888AACCAA90
:10023000444444444400EEEEAAAA00CCAAAAAA0070
:1002400044AAAA4400CCAACC880066AA66220088E8
:10025000EE88880066CC22CC44EE44444400AAAA2E
:10026000AA4400AAAA444400AAAAEEAA00AA4444A6
:10027000AA00AAAA66CC00EE66CCEE2244CC4422A8
:100280004444444444884466448800CCAA000000A6
:100290009EAAFED7ABCF18F0AECF01F018A202D0C5
:1002A000AB98AB880000000CF3DF0150120802E0AD
:1002B000000E01D0010E0201646F0001E9DF015060
:1002C000340802E0000E01D0010E02016415666FD1
:1002D0000001DEDF0150560802E0000E01D0010EE1
:1002E00002016615686F0001D3DF0150780802E053
:1002F000000E01D0010E020168156A6F0001C8DF0F
:100300000150900802E0000E01D0010E02016A15B2
:10031000D8A4FF009E9A00012CEF00F002015F516B
:10032000030803E19296898602D092988988949274
:100330008B92936A60C28AFF94948B84270E006E1E
:10034000002EFED70000000094948B94929689961C
:10035000929889980001000C02011C6B1C5107083F
:1003600044E394908B90030E5F6F400E606F00012A
:10037000D5DF040E02015F6F400E606F0001CEDF1B
:1003800002011C51B8091E6F030E5F6F1EC260F29E
:100390000001C4DF02011C51B8091E6F040E5F6F1B
:1003A0001EC260F20001BADF94908B8002011D6BC7
:1003B0001D513F0818E31B51FF0DF3CF1EF2030E32
:1003C0005F6F1EC260F20001A9DF02011B51FF0D29
:1003D000F3CF1EF2040E5F6F1EC260F200019EDFBB
:1003E00002011D2BE5D71C2BB9D700014FEF02F0FE
:1003F000929A898A94948B949296899692988998E5
:1004000094908B90030E02015F6FC00E606F00012D
:1004100085DF040E02015F6FC00E606F00017EDF9A
:10042000030E02015F6F400E606F000177DF040E64
:1004300002015F6F400E606F000170DF030E02016A
:100440005F6FB80E606F000169DF040E02015F6F1D
:10045000B80E606F000162DF02011A2D0FD0030E8B
:100460005F6F3F0E606F000159DF040E02015F6F86
:100470003F0E606F000152DF0ED00201030E5F6F6E
:100480003E0E606F00014ADF040E02015F6F3E0EF8
:10049000606F000143DF02011B6B00015DD7BBEF02
:1004A0000DF0006A016A02012951D8902AB1002694
:1004B000003201322AB30026003201322AB500266A
:1004C000003201322AB70026003201322AB9002652
:1004D000003201322ABB0026003201322ABD00263A
:1004E000003201322ABF0026003201320001000C26
:1004F00002015C51030803E19296898602D092982A
:100500008988FF0E936E94928B8294948B84270E2D
:10051000006E002EFED70000000094948B94270EEE
:10052000006E002EFED70000000094948B84270EEE
:10053000006E002EFED700000000FF0E936E81CFEC
:100540005DF294948B9492968996929889985DC264
:1005500001F00001D5EF02F0030E02015B6F57516D
:100560003F0804E2400E575F040E5B6F94908B903F
:10057000579F578D5BC25FF257C260F20001CEDE1B
:1005800002015831006E003200321F0E001600507A
:10059000BF0BB8095E6F5BC25FF2606F0001BEDE29
:1005A00094908B805BC25CF2A3D701C05AF2020127
:1005B000592D0FD05851070B5C6F010E006E5C5126
:1005C000016E04E0D8900036012EFCD700505A137B
:1005D0000FD05851070B5C6F010E006E5C51016E1D
:1005E00004E0D8900036012EFCD70050FF0A5A17BD
:1005F00094908B905BC25FF257C260F200018EDE76
:1006000094908B805BC25FF25AC260F287DE000C6E
:1006100002011A511C5D286F285128AF03D0000E2B
:10062000D8802855236F1B511D5D286F285128AF96
:1006300003D0000ED8802855246F1AC21FF21BC2A7
:1006400020F21A511C5D03E2FF0E216F02D0010E51
:10065000216F1B511D5D03E2FF0E226F02D0010EC0
:10066000226F2451800A006E2351800A005C01E051
:1006700051E2020E296F24C22AF2000112DF0201A8
:100680002351015C036AE8BE0306256F03C026F20E
:10069000276B23BF3ED02751235D3BE31FC257F298
:1006A00020C258F21EC259F2000156DF020126BFD5
:1006B00001D011D0020E296F24C22AF20001F1DE0E
:1006C0000150036AE8BE03060201252703502623D2
:1006D00021511F271CD0020E296F24C22AF20001CB
:1006E000E0DE01C028F2020E0201296F23C22AF2C5
:1006F0000001D7DE01500201285D036AE8BE03064F
:1007000025270350262321511F2722512027272B3D
:10071000C0D750D0020E296F23C22AF20001C1DED9
:1007200002012451015C036AE8BE0306256F03C081
:1007300026F2276B24BF3ED02751245D3BE31FC226
:1007400057F220C258F21EC259F2000105DF020121
:1007500026BF01D011D0020E296F23C22AF2000158
:10076000A0DE0150036AE8BE0306020125270350FC
:100770002623225120271CD0020E296F23C22AF2E1
:1007800000018FDE01C028F2020E0201296F24C28F
:100790002AF2000186DE01500201285D036AE8BEEC
:1007A000030625270350262321511F2722512027E6
:1007B000272BC0D70001C7EF0DF0020159515B0391
:1007C000F3CF01F0F4CF00F05C03F35000265A5150
:1007D0005B03F3500020026E0001000C02014E6B1F
:1007E000036A4E514B25E96E4C510320EA6EEF52DD
:1007F000D8B487D0036A4E514B25E96E4C51032083
:10080000EA6EEF501F0841E2036A4E514B25E96E34
:100810004C510320EA6EEF507E0837E3036A4E51D5
:100820004B25E96E4C510320EA6E200EEF5C586FA9
:100830005A6B596F5C6B050E5B6F0001BEDF02C027
:100840005AF2020101C059F2020EEA6E510EE96E2F
:1008500002C05EF201C05DF2F2CF5BF2F29E026A6C
:10086000050E016E022A5EC2F7FF5D51000116DC23
:100870000A000900EF6AF5CFEEFF012EFAD7022E2B
:10088000F8D702015BBFF28E05D0516B526B536BF0
:10089000546B556B030E49257F0803E2496B060E26
:1008A0004A27030E4F6F4F5329E0506B50510408F5
:1008B00021E3036A5051510FE96E020E0320EA6EE4
:1008C000EFCF56F256C200F04F51016E04E0D890BF
:1008D0000032012EFCD700A00BD050514A25566F94
:1008E00049C257F2586F4DC259F2000135DE02017C
:1008F000502BDCD74F514F07492BD5D74E2B492BC7
:100900006FD70001000C0201496B360E4A6F4C6B29
:100910004E0E4B6F010E4D6F000160DF1F2C0CD08F
:10092000080E0201496F360E4A6F4C6B500E4B6F2A
:100930004D6B000153DF1DD01F5002080CE1080E63
:100940000201496F360E4A6F4C6B540E4B6F4D6B64
:10095000000144DF0ED01F5003080BE1080E020116
:10096000496F360E4A6F4C6B5A0E4B6F4D6B000140
:1009700035DF1AC21FF01F2C09D01E0E236E8A0EFF
:10098000226E220E216E7B0E206E17D01F500208A1
:1009900009E1A40E236E8A0E226E220E216E7A0EBB
:1009A000206E0BD01F50030808E1980E236E890EAD
:1009B000226E220E216E790E206E1F2C0DD0080E95
:1009C0000201496F360E4A6F4C6B500E4B6F010E91
:1009D0004D6F000103DF1FD01F5002080DE1080E0C
:1009E0000201496F360E4A6F4C6B540E4B6F010E6D
:1009F0004D6F0001F3DE0FD01F5003080CE1080E0D
:100A00000201496F360E4A6F4C6B5A0E4B6F010E46
:100A10004D6F0001E3DE09EF0EF08E0E006E2AC26C
:100A200001F029C202F0036A015209E102C001F09B
:100A3000026A080E005E015202E1006A08D0D890F6
:100A400001BE04D0023601360006F9D7019E00002F
:100A5000000C02012951D8B4A5D0356F2D51D8B45E
:100A6000A1D0355F05E37F0E3527D8B09BD006D0E7
:100A7000810E355FD8A096D0D8B494D035C200F09E
:100A8000016A026A036A346B2AC233F2338F2BC2C3
:100A900032F22CC231F2190E356F3051315F0DE256
:100AA000010E325F0AE2335F08E2345F06E2342B64
:100AB000332B322B3051312728D02F51325F12E2A5
:100AC000010E335F0FE2345F0DE2342B332B2F51D5
:100AD00032273051312719E3322B17E1332B15E13F
:100AE000342B13D02E518009335F0EE2010E345F98
:100AF0000BE2342B2E51800933272F513227E9E3A3
:100B0000332BE7E1342BE5D70380352F01D00BD011
:100B1000D8903137323733373437D89003360236EE
:100B200001363637BAD736A106D0D8900132023214
:100B30000332363302D0000635E036BF1ED0D890DF
:100B400031373237333734373051315F07E2010EF6
:100B5000325F04E2335F02E2345F1AE32F51325F07
:100B600005E2010E335F02E2345F12E32E51800989
:100B7000335F03E2010E345F0BE3032A09E1022A2B
:100B800007E1012A05E1002A0DE0013202320332B9
:100B90002AC235F22E51351B35AF02D0018E06D058
:100BA000019E04D0006A016A026A036A0000000123
:100BB000000C02015651D8B471D0006E5A51D8B40D
:100BC0006DD0002604E3810E002668E204D07F0E7B
:100BD000005E64E363E057C25EF25B515E1B578FB9
:100BE0005B8F59515D03F4CF60F258515C03F4CF31
:100BF00003F0F3CF5FF25D03F3506027F4505F23FF
:100C0000000E032259515C03F3506027F4505F2318
:100C1000000E026A0322022257515D03F3505F2740
:100C2000F4500322000E022257515C03F3500326B6
:100C3000F4500222000E016A012259515B03F35065
:100C40005F27F4500322000E0222012258515B0359
:100C5000F3500326F4500222000E012257515B0389
:100C6000F3500226F4500122002A01BE05D05F375E
:100C70000336023601360006000E5FAF0AD0032AA3
:100C800002220122015005E1025003E1035001E17B
:100C9000002A5EBF018E5EAF019E04D0006A016A29
:100CA000026A036A00000001000C02015651B608F6
:100CB000566F036A57C25AF2578FD890573358333A
:100CC00059330332023201320032562FF6D75AAF6F
:100CD0000BD0001E011E021E031E002AD8B4012ADA
:100CE000D8B4022AD8B4032A00012BEF08F0006A16
:100CF000016A026A036A02015E6B5F6B606B616B83
:100D00005D515C115B115A112CE0200E626FD8907E
:100D100056375737583759375E375F37603761373F
:100D20005D51615D08E15C51605D05E15B515F5DB6
:100D300002E15A515E5D0FE35A515E5F5B51D8A0EC
:100D40005B3D5F5F5C51D8A05C3D605F5D51D8A0AA
:100D50005D3D615FD8800036013602360336622F72
:100D6000D6D70000020EEA6E5E0EE96E0001000C9E
:100D70001AC0EAFF19C0E9FF020156C2EFFFE92AD3
:100D8000D8B4EA2AEF6A192AD8B41A2A0001000C4A
:100D9000020E1A6E370E196E890EE96E32C24CF2CF
:100DA00031C24BF230C24AF22FC249F2060E0201A2
:100DB0004D6F000125D9020E1A6E400E196E890E74
:100DC000E96E36C24CF235C24BF234C24AF233C23B
:100DD00049F2060E02014D6F000112D902013B6B70
:100DE000446B2DC249F22EC24AF2020E4C6F370EEE
:100DF0004B6F4D6B0001F2DC2DC249F22EC24AF25C
:100E0000020E02014C6F400E4B6F010E4D6F000140
:100E1000E5DC000C020EEA6E1A0EE96EEF500EE0F1
:100E20000F0E016E006A002EFED7012EFBD78F0E2B
:100E3000006E002EFED70000EF2EF2D7000C010E40
:100E400002011B5F0EE3020EEA6E1B0EE96EEF500D
:100E500008E0020E006E002EFED700000000EF2E0C
:100E6000F8D7000102EF0FF08E0E006E02011E5146
:100E7000005E1FC202F020C201F0028E005209E0A3
:100E8000D890025202E1015204E002320132002EF7
:100E9000F7D71FAF05D0011E021E012AD8B4022ABF
:060EA00000000001000C3F
:10100000E95002014E6F4D51506F1BE04CC259F236
:101010004BC258F24AC257F249C256F25D6B5C6B42
:10102000200E5B6F820E5A6F0001C3DD03C04CF2CD
:1010300002C04BF201C04AF200C049F20201502F37
:10104000E5D74CC259F24BC258F24AC257F249C2D4
:1010500056F200012AD603C04CF202C04BF201C086
:101060004AF200C049F202014CAF0DD04E074E8B40
:10107000491F4A1F4B1F4C1F492BD8B44A2BD8B4C9
:101080004B2BD8B44C2B3B0E556F9A0E546FCA0E97
:10109000536F526B0A0E506F4D51D8B44E2B4CC249
:1010A00059F24BC258F24AC257F249C256F255C2DF
:1010B0005DF254C25CF253C25BF252C25AF20001BA
:1010C00016DE0150EFCF49F2ECCF4AF2ECCF4BF2F3
:1010D000ECCF4CF2005213E102014D29505DD8A42F
:1010E00002D000010CD04E510DE00F0B505D01E01D
:1010F00040E24EBF3ED04EBD05D0200E34D0200E73
:1011000002014E174EAB0ED04E9B4D51D8A44E0748
:1011100000504E6F2D0E566F00012ADE02014E5117
:10112000006E4E6B4D51505D0CE100504E6F2E0E17
:10113000566F00011DDE02014E51006E200E4E174B
:10114000000E300E4EAB0FD04E9B4D51D8A44E0723
:1011500000504E6F2D0E566F00010ADE02014E51F7
:10116000006E4E6B300E002600C056F2000100DE0D
:10117000020155C259F254C258F253C257F252C238
:1011800056F25D6B5C6B5B6B0A0E5A6F0001AFDD54
:1011900003C055F202C054F201C053F200C052F233
:1011A0000201502F7CD70001000C02011D6B1E6B49
:1011B0001F6B206B216B226B236B246B496B240EFE
:1011C0004A6F4C6B410E4B6F010E4D6F0001EEEC00
:1011D00003F002011A2D74D01E50190DF3502A6B22
:1011E000296F00011ADC03C020F202C01FF201C007
:1011F0001EF200C01DF21CC25AF21BC259F20201BB
:101200005C6B190E5B6F0001DDEC03F002C02AF28B
:1012100001C029F2000101DC03C024F202C023F264
:1012200001C022F200C021F220C22CF21FC22BF218
:101230001EC22AF21DC229F20201306B2F6B7A0EF8
:101240002E6F880E2D6F000104DC00C025F201C056
:1012500026F202C027F203C028F224C22CF223C2D5
:101260002BF222C22AF221C229F20201306B2F6B2B
:101270007A0E2E6F880E2D6F000129EC05F000C04C
:1012800029F201C02AF202C02BF203C02CF20C0E8C
:1012900002012D6F240E2E6F28C232F227C231F2C6
:1012A00026C230F225C22FF22CC236F22BC235F202
:1012B0002AC234F229C233F200016ADD45D00201AC
:1012C0001A51020842E11E50190DF3502A6B296F82
:1012D00000010DEC05F000C025F201C026F202C0AD
:1012E00027F203C028F21CC25AF21BC259F20201B3
:1012F0005C6B190E5B6F0001DDEC03F002C02AF29B
:1013000001C029F200010DEC05F000C029F201C076
:101310002AF202C02BF203C02CF20C0E02012D6F38
:10132000240E2E6F28C232F227C231F226C230F2CA
:1013300025C22FF22CC236F22BC235F22AC234F269
:1013400029C233F2000124DD02011AC21DF01BC2C2
:101350001EF01A2D05D01E500F0802E3100E1E6E4F
:10136000040E496F2A0E4A6F4C6B440E4B6F010EF0
:101370004D6F0001EEEC03F012EF0EF002011C6B5A
:101380001D6B1E6B1F6B1C30006E00323F0E001673
:1013900000502A6B296F00010DEC05F003C059F2D3
:1013A00002C058F201C057F200C056F223C05DF2ED
:1013B00022C05CF221C05BF220C05AF2D9EC05F0E9
:1013C00003C01FF202C01EF201C01DF200C01CF2D9
:1013D00002011A530DE10C0E496F180E4A6F4C6B47
:1013E000330E4B6F4D6B0001EEEC03F098D0020111
:1013F0001A2D4AD00C0E496F180E4A6F4C6B370EDF
:101400004B6F4D6B0001EEEC03F002011B31006EDF
:1014100000323F0E001600502A6B296F00010DECC0
:1014200005F003C059F202C058F201C057F200C0E3
:1014300056F223C05DF222C05CF221C05BF220C0F4
:101440005AF2D9EC05F000C021F201C022F202C02C
:1014500023F203C024F20C0E02012D6F1E0E2E6F1C
:101460001FC232F21EC231F21DC230F21CC22FF274
:1014700003C036F202C035F201C034F200C033F2CC
:10148000000186DC4CD002011A51020849E10C0E21
:10149000496F180E4A6F4C6B3C0E4B6F4D6B000141
:1014A000EEEC03F002011B31006E00323F0E00161D
:1014B00000502A6B296F00010DEC05F003C059F2B2
:1014C00002C058F201C057F200C056F223C05DF2CC
:1014D00022C05CF221C05BF220C05AF2D9EC05F0C8
:1014E00000C021F201C022F202C023F203C024F2A4
:1014F0000C0E02012D6F1E0E2E6F1FC232F21EC285
:1015000031F21DC230F21CC22FF203C036F202C00B
:1015100035F201C034F200C033F2000139DC0201BF
:101520001AC21BF01BC21CF0496B180E4A6F4C6BA1
:10153000300E4B6F010E4D6F0001EEEC03F01B52AD
:101540000EE10C0E0201496F180E4A6F4C6B330E00
:101550004B6F010E4D6F0001EEEC03F020D01B2C01
:101560000ED00C0E0201496F180E4A6F4C6B370EED
:101570004B6F010E4D6F0001EEEC03F010D01B50CD
:1015800002080DE10C0E0201496F180E4A6F4C6BF8
:101590003C0E4B6F010E4D6F0001EEEC03F01AEFA5
:1015A0000EF0EACF34F2E9CF33F202012D39F0091F
:1015B0002F6F2F27E20F306F320F326F2D510F0B2D
:1015C000302730273227E90F316F312731272C3967
:1015D0000F0B3127322731373237321F32372C5138
:1015E0000F0B32272F37070E2E6F0A0E31073227C7
:1015F000FDE330073127FDE32F073027FDE32E07FA
:101600002F27FDE3020EEA6E2E0EE96E070E33154C
:10161000339DE926320EE95CD8B4338DEF50006E6D
:1016200008E133BD06D033B916D033B702D0200E4F
:1016300003D033873399300E0026EACF2DF2E9CF5D
:101640002CF200C056F20001B8EC06F02DC2EAFF01
:101650002CC2E9FF0201EE5033ADDCD70001000CD3
:10166000020E1A6E200E196E100EE96E1DC22DF2BA
:101670001CC22CF296DF020E1A6E260E196E100E88
:10168000E96E1FC22DF21EC22CF28BDF0201256B08
:101690002B6B1AC249F21BC24AF2020E4C6F200E8B
:1016A0004B6F4D6B0001EEEC03F01AC249F21BC206
:1016B0004AF2020E02014C6F260E4B6F010E4D6F67
:1016C0000001EEEC03F063EF11F0800ED8A202D01F
:1016D0000201211B0201266B276B1DC225F221513D
:1016E000251B1C51D8B4DFD0246F006E2051D8B414
:1016F000E3D0245FD8B483D03EE321C22AF22A8FFC
:1017000022C229F223C228F2276BD8902A33293328
:1017100028332733242FF8D725AF03D02681E0D0F4
:10172000269124912689020EEA6E1F0EE96EEBD0F7
:10173000269925BF0AD024A113D02A332933283370
:101740002733002AD8B4C7D00BD02ABF0CD0D890EA
:101750002737283729372A370006D8B4BCD0F5D721
:10176000268D6DD0269D1DC225F21DAF02D02A8F79
:10177000ABD02A9FA9D020C224F220C200F01C5175
:10178000245F1DC22AF22A8F1EC229F21FC228F22C
:10179000276BD8902A33293328332733242FF8D7BF
:1017A00025AF03D026839CD026932491268B020E4E
:1017B000EA6E230EE96EA7D0269B25BF0AD024A18E
:1017C00013D02A33293328332733002AD8B483D0BF
:1017D0000BD02ABF0CD0D8902737283729372A3783
:1017E0000006D8B478D0F5D7268F29D0269F21C2FD
:1017F00025F221AF02D02A8F67D02A9F65D021C25F
:101800002AF22A8F22C229F223C228F225AF04D05D
:101810002A9F268565D02695276B2491020EEA6EB5
:101820001F0EE96E70D025BF1CD01DC225F224A169
:1018300006D02A33293328332733002A4CE027AF38
:101840000BD0282B09E1292B07E12A2B05E12A33AC
:1018500029332833002A3FE026BD84D726BFC6D7C8
:101860001CD0800E2A1B2AAF04D03AD021C225F208
:101870000AD01DC225F22A5306E1295304E1285358
:1018800002E1006A21D02ABF08D0D8902737283734
:1018900029372A37002EF7D71ED025AF02D02A8F3E
:1018A00013D02A9F11D020C200F021C22AF222C2F6
:1018B00029F223C228F208D01CC200F01DC22AF26D
:1018C0001EC229F21FC228F22AC201F029C202F068
:1018D00028C203F034D0006A016A026A036A2FD07A
:1018E000276B281F291F2A1F271F272B05E1282BBD
:1018F00003E1292B01E12A2B26B112D726B354D7B5
:1019000026B589D7B3D7EF50282705E3292B03E164
:101910002A2BD8B42481ED52EF50292703E32A2B38
:10192000D8B42481ED52EF50EFBE01D0800A2A27AF
:10193000D8B0248126B9FCD626BB3ED774D7000088
:101940000001000C1CC223F202012051231B23AF13
:1019500005D0D894D8901CBFD8802FD01CC223F2B9
:101960001FC224F21B51245F06E023AF26D0D850BB
:10197000010AD86E22D020C224F21C51245F06E056
:1019800023AF1BD0D850010AD86E17D021C224F241
:101990001D51245F06E023AF10D0D850010AD86E45
:1019A0000CD022C224F21E51245F06E023AF05D0E2
:1019B000D850010AD86E01D0D8900001000CF86A06
:1019C000D09E0D8EEA6AE96AB896190EAF6E260EA1
:1019D000AC6E900EAB6EC150C00B0F09C16E070EFE
:1019E000B46E186A196A1A6A1B6A7F0E1C6E010EA1
:1019F0001D6E040E1E6E010E1F6E7B0E206E220EDB
:101A0000216E8A0E226E1E0E236E410E246E760EFD
:101A1000256E266A4D0E276E780E286E296A4D0EA9
:101A20002A6E6E0E2B6E2C6A500E2D6E2E6E2F6A45
:101A3000540E306E680E316E326A4F0E336E660E83
:101A4000346E356E366A520E376E690E386E730E0E
:101A5000396E650E3A6E3B6A460E3C6E610E3D6E07
:101A60006C0E3E6E3F6E406A540E416E6D0E426EBD
:101A7000436A446E730E456E2F0E466E640E476EBB
:101A8000690E486E760E496E4A6A480E4B6E7A0EA3
:101A90004C6E4D6A520E4E6E4F6A300E506E2D0EC9
:101AA000516E350E526E536A300E546E2D0E556EB9
:101AB000320E566E2E0E576E350E586E596A300E17
:101AC0005A6E2D0E5B6E310E5C6E2E0E5D6E320EFA
:101AD0005E6E5F6A0101F06B010EF16FF26BF36BEA
:101AE000F46BF56BF66BF76BF86BF96BFA6BFB6BE2
:101AF000FC6BFD6BFE6BFF6B0201006B016B026BFD
:101B0000036B046B056B066B076B086B096B0A6B49
:101B10000B6B0C6B0D6B0E6B0F6B106B116B126BF9
:101B2000136B146B156B166B176B186B196BC1501D
:101B3000C00B0E09C16EC090C082C084C08EC2802E
:101B4000880ED56ECD6A000ECA6E7F0ECB6EB15078
:101B5000480BB16EB70EB1169484BD6ABD6AB1165A
:101B60009482BA6ABA6A9D8AC00EF212010E1A6F86
:101B70000001F8EF01F01C0E02011A6F1B6B1C6FC5
:101B80003F0E1D6F010E1E6F000108EF03F00201F2
:101B9000496B4A6B4C6B240E4B6F010E4D6F00016D
:101BA000EEEC03F00201496B060E4A6F4C6B270EF8
:101BB0004B6F010E4D6F0001EEEC03F00201496B1B
:101BC0000C0E4A6F4C6B2A0E4B6F010E4D6F0001CD
:101BD000EEEC03F00201496B120E4A6F4C6B2D0EB6
:101BE0004B6F010E4D6F0001EEEC03F0140E02017D
:101BF000496F300E4A6F4C6B4B0E4B6F010E4D6FA1
:101C00000001EEEC03F0010E02011A6F000183EFF8
:101C100004F0010E02011A6F1C6B140E1B6F000101
:101C2000D5EF08F0010E02011A6F7F0E1B6F000145
:101C3000BEEF09F0000E016EC250C30B0110C26E60
:101C40000A0E02011A6F00010AEC07F0640E02018D
:101C50001A6F00010AEC07F01F2C0FD002011B6B5A
:101C60001C340101F26F02011B350101F36FF237E1
:101C7000F337FC0EF21717D000011F5002080CE1D9
:101C800002011B6BD8901C340101F26F02011B355D
:101C90000101F36F08D000011F50030805E10101A5
:101CA000F36B1CC0F2F100011B2C46D00101F56B57
:101CB000F46BC282C2B2FED7C4CF1BF2C3CF1AF2FA
:101CC0000101F3510201C45C14E307E11A5101015F
:101CD000F25DD8A002D002010CD00101F43D05D084
:101CE000F53D03D0020105D00101F42BD8B4F52B4A
:101CF000E0D70101F56BF46BC282C2B2FED7C4CF4C
:101D00001BF20201C3CF1AF2C4500101F35D12E3CA
:101D100008E1F25102011A5DD8A002D001010AD0F7
:101D20000101F43D03D0F53D01D004D0F42BD8B42B
:101D3000F52BE2D747D000011B50020845E1010115
:101D4000F56BF46BC282C2B2FED7C4CF1BF20201A4
:101D5000C3CF1AF2C4500101F35D12E308E1F2515E
:101D600002011A5DD8A002D001010AD00101F43DA0
:101D700003D0F53D01D004D0F42BD8B4F52BE2D735
:101D8000F56BF46BC282C2B2FED7C4CF1BF2C3CFD5
:101D90001AF20101F3510201C45C15E307E11A5183
:101DA0000101F25DD8A002D002010DD00101F43D85
:101DB00005D0F53D03D0020106D00101F42BD8B4C3
:101DC000F52BE0D7020100011D2C21D00101F06BA1
:101DD000F05163081AE3D890F035036A600FE96E9A
:101DE000000E0320EA6EC282C2B2FED7C3CFEFFF5D
:101DF000C4CFECFF100E1E5C02011A6F1B6F0001B6
:101E00001FEF07F00101F02BE3D720D000011D5098
:101E100002081CE10101F06BF051630817E3D89050
:101E2000F035036A600FE96E000E0320EA6EC2828D
:101E3000C2B2FED7C3CFEFFFC4CFECFF1EC01AF271
:101E400000010AEC07F00101F02BE6D70101F06B6D
:101E5000F0516308D8A099D01F2C32D0036AF051FA
:101E6000280F016E010E0322020103C01BF2D8905D
:101E70000101F035036A600FE96E000E0320EA6E7F
:101E8000ECCF1DF2ED52EFCF1CF202011D31036EBB
:101E90001C31026E0332023203320232033202324A
:101EA0000F0E03160250FF0A400F006E000E03567D
:101EB0001BC2EAFF01C0E9FF00C0EFFF63D00101D0
:101EC0001F50020830E1036AF051280F016E010E25
:101ED0000322020103C01BF2D8900101F035036A0E
:101EE000600FE96E000E0320EA6EECCF1DF2ED529A
:101EF000EFCF1CF202011D31036E1C31026E033262
:101F00000232033202321F0E03160250FF0A400F44
:101F1000006E000E03561BC2EAFF01C0E9FF00C0BD
:101F2000EFFF30D001011F5003082DE1036AF0518B
:101F3000280F016E010E0322020103C01BF2D8908C
:101F40000101F035036A600FE96E000E0320EA6EAE
:101F5000ECCF1DF2ED52EFCF1CF202011D31036EEA
:101F60001C31026E033202323F0E03160250FF0A8A
:101F7000400F006E000E03561BC2EAFF01C0E9FFCE
:101F800000C0EFFF0101F02B63D7010EF06FF0519D
:101F900063081AE31C0EF02502011A6F036A01019F
:101FA000F0518C0FE96E010E0320EA6EEFCF1BF2A9
:101FB0001AC257F21BC258F20201596B0001ACEC75
:101FC00002F00101F02BE3D7010EF06FF05163082E
:101FD0001BE31C0EF02502011A6F036A0101F05188
:101FE000280FE96E010E0320EA6EEFCF1BF21AC232
:101FF00057F21BC258F2010E0201596F0001ACECFE
:1020000002F00101F02BE2D7F06BF05163081DE301
:10201000036AF0518C0F016E010E0322020103C00E
:102020001BF2036A0101F051280FE96E010E032033
:10203000EA6EEFCF1CF202011BC2EAFF01C0E9FF0A
:102040001CC2EFFF0101F02BE0D71B52D8B440D1E6
:10205000F06BF0513E080FE31C0EF12502011A6FE0
:10206000576FF0C158F2596B0001ACEC02F0030E4F
:102070000101F027EED71B2C42D0010EF16F036A4D
:10208000F151280FE96E010E0320EA6EEFCF1AF22C
:102090001C30006E00323F0E00160050FF0A400F49
:1020A00002011A5D09E20101F1516208D8B002D0C3
:1020B000020102D0F12BE3D70101F12B036AF151A8
:1020C000280FE96E010E0320EA6EEFCF1AF21C30E2
:1020D000006E00323F0E00160050FF0A400F020152
:1020E0001A5D0BE00AE30101F1516208D8B002D099
:1020F000020103D0F12BE2D7020144D001011B50B1
:1021000002083FE1010EF16F036AF151280FE96EF9
:10211000010E0320EA6EEFCF1AF21C30006E00327F
:102120003F0E00160050FF0A400F02011A5D0AE040
:1021300009E30101F1516208D8B002D0020102D0D6
:10214000F12BE2D70101F12B036AF151280FE96E5F
:10215000010E0320EA6EEFCF1AF21C30006E00323F
:102160003F0E00160050FF0A400F02011A5D0AE2FE
:102170000101F1516208D8B002D0020103D0F12B65
:10218000E3D702010101F06BF0513E0810E31C0E91
:10219000F12502011A6F576FF0C158F2010E596F05
:1021A0000001ACEC02F0030E0101F027EDD70201B3
:1021B0001B6BF1C11AF21BC25AF2F1C159F25C6BEE
:1021C0001EC05BF20001DDEC03F002C0F5F101C0BE
:1021D000F4F11D2C40D0F5C12AF2F4C129F20DEC26
:1021E00005F002012C6B2B6B7A0E2A6F880E296F7B
:1021F00003C030F202C02FF201C02EF200C02DF257
:10220000000129EC05F000C01AF201C01BF202C067
:102210001CF203C01DF203C059F202C058F201C003
:1022200057F200C056F202015D6B5C6B7A0E5B6F79
:10223000880E5A6F0001D9EC05F003C021F202C0EC
:1022400020F201C01FF200C01EF234EC07F002C001
:1022500017F201C016F21D50020826E1F5C12AF25C
:10226000F4C129F20DEC05F002012C6B2B6B7A0EF8
:102270002A6F880E296F03C030F202C02FF201C00E
:102280002EF200C02DF2000129EC05F003C021F26E
:1022900002C020F201C01FF200C01EF234EC07F0B1
:1022A00002C017F201C016F202011A6B300E1B6F4A
:1022B00019C21DF218C21CF217C21FF216C21EF27A
:1022C000000130EF0BF017C219F216C218F201012B
:1022D000F96BF86BF76BF66BF06BF051630834E356
:1022E000036AF051280FE96E010E0320EA6EEF50E9
:1022F00002012A6B296F00010DEC05F0EACF1BF2F9
:10230000E9CF1AF2D892F9C11FF2F8C11EF2F7C153
:102310001DF2F6C11CF203C023F202C022F201C07A
:1023200021F200C020F265EC0BF01BC2EAFF1AC2DA
:10233000E9FF03C0F9F102C0F8F101C0F7F100C0F4
:10234000F6F10101F02BC9D7F9C12CF2F8C12BF23B
:10235000F7C12AF2F6C129F20201306B2F6B480E49
:102360002E6F850E2D6F000129EC05F0D882020139
:102370001F6B1E6B7C0E1D6F840E1C6F03C023F23F
:1023800002C022F201C021F200C020F2000165EC7F
:102390000BF000C01AF201C01BF202C01CF203C015
:1023A0001DF203C059F202C058F201C057F200C03A
:1023B00056F223C05DF222C05CF221C05BF220C065
:1023C0005AF2D9EC05F003C0F9F102C0F8F101C0EE
:1023D000F7F100C0F6F10C0E02012D6F2E6BFDC15E
:1023E00032F2FCC131F2FBC130F2FAC12FF2F9C175
:1023F00036F2F8C135F2F7C134F2F6C133F200011A
:10240000C8EC06F0F9C1FDF1F8C1FCF1F7C1FBF130
:10241000F6C1FAF10201016B006B7C0E0101FF6F46
:10242000840EFE6FF06BF05163083BE3036AF051DA
:10243000280FE96E010E0320EA6E02012A6BEFCF2E
:1024400029F200010DEC05F003C01EF202C01DF2DE
:1024500001C01CF200C01BF201C222F200C221F234
:10246000FFC120F2FEC11FF2A2EC0CF017E3036AD9
:102470000101F051280FE96E010E0320EA6EEF50C2
:1024800002012A6B296F00010DEC05F003C001F277
:1024900002C000F201C0FFF100C0FEF10101F02B0B
:1024A000C2D7D88202011F6B1E6B7C0E1D6F840E7B
:1024B0001C6F01C223F200C222F2FFC121F2FEC151
:1024C00020F2000165EC0BF000C01AF201C01BF213
:1024D00002C01CF203C01DF203C059F202C058F240
:1024E00001C057F200C056F223C05DF222C05CF278
:1024F00021C05BF220C05AF2D9EC05F003C001F212
:1025000002C000F201C0FFF100C0FEF10C0E02019A
:102510002D6F060E2E6F05C232F204C231F203C2D5
:1025200030F202C22FF201C236F200C235F2FFC110
:1025300034F2FEC133F20001C8EC06F001C205F22C
:1025400000C204F2FFC103F2FEC102F20201096BF4
:10255000086B076B066B0101F06BF05163083BE3FE
:10256000036AF051280FE96E010E0320EA6E0201A2
:102570002A6BEFCF29F200010DEC05F009C21EF223
:1025800008C21DF207C21CF206C21BF203C022F2EF
:1025900002C021F201C020F200C01FF2A2EC0CF038
:1025A00017E3036A0101F051280FE96E010E0320C1
:1025B000EA6EEF5002012A6B296F00010DEC05F065
:1025C00003C009F202C008F201C007F200C006F21F
:1025D0000101F02BC2D7D88202011F6B1E6B7C0E4B
:1025E0001D6F840E1C6F09C223F208C222F207C2BB
:1025F00021F206C220F2000165EC0BF000C01AF2D5
:1026000001C01BF202C01CF203C01DF203C059F24C
:1026100002C058F201C057F200C056F223C05DF26A
:1026200022C05CF221C05BF220C05AF2D9EC05F066
:1026300003C009F202C008F201C007F200C006F2AE
:102640000C0E02012D6F2E6F0DC232F20CC231F250
:102650000BC230F20AC22FF209C236F208C235F2BA
:1026600007C234F206C233F20001C8EC06F009C218
:102670000DF208C20CF207C20BF206C20AF2D882AF
:1026800001C21FF200C21EF2FFC11DF2FEC11CF208
:1026900009C223F208C222F207C221F206C220F2C6
:1026A00065EC0BF003C011F202C010F201C00FF292
:1026B00000C00EF20C0E02012D6F120E2E6F15C20D
:1026C00032F214C231F213C230F212C22FF211C22E
:1026D00036F210C235F20FC234F20EC233F20001EC
:1026E000C8EC06F011C215F210C214F20FC213F2B8
:1026F0000EC212F21B521CE01D0E0101F06FF051D0
:102700007E0816E31C30006E00323F0E00160050AB
:10271000FF0A400F02011A6FF0C157F2586F010E05
:10272000596F0001ACEC02F0030E0101F027E7D76E
:102730000101F06BF0513E082CE3350E0201576F9A
:10274000F0C158F2010E596F0001ACEC02F04E0ED0
:102750000201576FF0C158F2010E596F0001ACEC45
:1027600002F0670E0201576FF0C158F2010E596F67
:102770000001ACEC02F07F0E0201576FF0C158F27D
:10278000010E596F0001ACEC02F0050E0101F027BB
:10279000D1D7640E02011A6F00010AEC07F02CEF8A
:0427A0000EF0030034
:020000040030CA
:0E000000240E3F1E008381000FC00FE00F4052
:00000001FF
